:100000002030840027300C208316FF2390008301CA
:10001000F92A04068001840A0406031D09286400E5
:020020000034AA
:1005F200831212232823FB2AAB01AC010310AA0C9D
:10060200A90C031C0B2B2708AB0728080318280A80
:10061200AC070310A70DA80D29082A0403190034FA
:10062200FF2A8B010730831299000330831685005D
:1006320083128501831681179F011F179F121F16B0
:100642001F149F1483129F171F131F140800831275
:100652006F232008A400492B05162208A5002308B1
:10066200A60025080319A603A503250A0319260ACD
:10067200031D322B05122208A5002308A600250817
:100682000319A603A503250A0319260A031D402BF5
:10069200A403240F2D2B2008A4006B2B85162208FF
:1006A200A5002308A60025080319A603A503250A09
:1006B2000319260A031D542B85122208A5002308BC
:1006C200A60025080319A603A503250A0319260A6D
:1006D200031D622BA403240F4F2B080083129F11CA
:1006E2001F110C139F149F18742BFF30A900AA012D
:1006F2001E08A700A801FD2283161E082B078312DD
:10070200A0002C0803182C0AA1009F111F150C131E
:100712009F149F188A2BFF30A900AA011E08A70068
:10072200A801FD2283161E082B078312A2002C08A3
:1007320003182C0AA300003021026430031920029E
:1007420064300318A62BA000A101A900AA01200869
:10075200A7002108A800C5232B08A0002C08A1008F
:10076200003023023230031922020318BB2B32302D
:0E077200A200A3010310A20DA30D0310A20DFF
:10078000A30D0310A20DA30D0800AD01AB01AC0138
:1007900029082A04031DCF2BA701A80100341F300C
:1007A000AD040310AD0AA90DAA0D031CD22BAA0C8F
:1007B000A90C2A082802031DDF2B29082702031C85
:1007C000E72B2908A7022A08031C2A0AA802AB0D56
:1007D000AC0DAD0BAD1AD72BAD1FF32BAB09AB0A8C
:1007E0000319AC03AC092B08A9002C08AA002D1F83
:0E07F0000034A709A70A0319A803A8090034BA
:02400E00C43FAD
:00000001FF
